:020000020000FC
:100000000C94E0040C942A000C942A000C942A000E
:100010000C942D010C942A000C942A000C942A00B4
:100020000C942A000C942A000C942A000C942A00A8
:100030000C942A000C947E020C942A000C942A0042
:100040000C942A000C942A000C942A000C942A0088
:100050000C942A00189519BC0E00669C0F00098AA2
:100060001000CE8511008B90120025AB13008DD6A9
:100070001400C2131600D4631700E3C718001D4113
:100080001A00C5D01B0031781D00010101010101DA
:100090000101010101010101010202020202020249
:1000A000020202030303030303030404040404051C
:1000B0000505050606060707070708080909090ACE
:1000C0000A0B0B0C0C0D0E0E0F1010111213131443
:1000D00015161718191A1C1D1E1F21222426272940
:1000E0002B2D2F313335383A3D3F4245484C4F5246
:1000F000565A5E62676B70757A7F858B91989EA564
:10010000ADB5BDC5CED7E0EAF5FF0DC7C59A5778A6
:10011000915DC1489138FC2B3322971AAD1413100E
:10012000800CB8098F07E00592048D03C3022602F4
:10013000AB014C010201C9009C0079005E0049003E
:1001400039002C0023001B001300000000010101F6
:100150000101020202020303030303040404040571
:100160000505050606060607070707080808080923
:100170000909090A0A0A0B0B0B0B0C0C0C0D0D0DCF
:100180000E0E0E0F0F0F101010111112121213136A
:1001900014141415151616171717181819191A1AF2
:1001A0001B1B1C1C1D1D1E1E1F1F20212122222364
:1001B000232425252627272829292A2B2B2C2D2DBA
:1001C0002E2F303031323333343536373838393AF0
:1001D0003B3C3D3E3F3F4041424344454647484902
:1001E0004A4B4C4D4E5051525354555657595A5BE9
:1001F0005C5D5F60616264656668696A6C6D6E70A3
:100200007173747677787A7B7D7E80828385868829
:100210008A8B8D8E9092949597999A9C9EA0A2A479
:10022000A5A7A9ABADAFB1B3B5B7B9BBBDBFC1C38E
:10023000C5C7C9CBCED0D2D4D6D9DBDDE0E2E4E766
:10024000E9EBEEF0F3F5F7FAFCFFE0E0E0E0E0E0E8
:10025000E0E0E0E4E8ECF0F4F8FC0F930FB70F9364
:100260001F932F933F934F935F936F937F93EF93DE
:10027000FF930F921F92509177007091780075FF55
:100280000CC01091BE0043FC109544FC109546FC38
:10029000109547FC1095110F3BC0142D77FF2CC013
:1002A00076FF4091D70076FD4091D60070FF1CC0CC
:1002B0006091D400EEE5F5E1E10FF61FC895042F3B
:1002C000010F102DEEE5F5E1E00FF61FC8950027B0
:1002D00010190809140F081D14F410E000E00023A1
:1002E00009F01FEF105814C0141718F01FEF105822
:1002F0000FC010E010580CC0142D70FF08C06091A2
:10030000D400EEE5F5E1E10FF61FC895102D105869
:100310006091D50070FF60E0072D73FF07C0EEE528
:10032000F1E2E00FF61FC895002D06C0EEE5FDE2F4
:10033000E00FF61FC895002D005855FD10270093BB
:10034000D8006FE71603F00172FF012F0603E00DDE
:10035000F11D8F01159507951595079578010919D8
:100360001A0913F401E010E86091DD004091890062
:100370005FEF541B569528E0520F651B08F460E0B0
:10038000492D5A2D3091DF002091DE00421B530B86
:1003900013F441E050E82091770024FF02C09A0155
:1003A00013C02091E0002223D1F356039001469F11
:1003B000210D381D001C08F423958894220F331F4B
:1003C0008894220F331F9901020F131F13F40FEFAC
:1003D0001FE7409189002091770024FD40918A0019
:1003E00014039001049F210D381D001C08F423956F
:1003F000920EA31E23F42FEF3FE7922EA32E3A2D49
:10040000292DE091DE00F091DF002E1B3F0B13F44D
:1004100021E030E8409189002091770024FD40914F
:100420008A0034039001249F210D381DE20FF31F31
:1004300013F4EFEFFFE7E093DE00F093DF000E2F01
:100440001F2F2091770024FF03C0E01AF10A8701D3
:10045000F80120918B002F3F29F01203F001029F39
:10046000E10DF81D939AF0589298F5BB9398939AE2
:10047000929AE5BB9398939AEEECF0E00191200EEE
:100480000191301E0191401E0191500E0191601E9C
:100490000191701EE0917800E5FD21C0E2FF1FC0D0
:1004A000E0917700E1FF10E0E1FD1FEF1123B9F0CB
:1004B0000091D800010390010091CE001127300374
:1004C000110B210C311E411E0091CF003003200C76
:1004D000311C411E0091D0003003300C411C1F9094
:1004E0000F90FF91EF917F916F915F914F913F91AD
:1004F0002F911F910F910FBF0F9118950F930FB769
:100500000F930CB1579878941F930023F2F4102F97
:10051000107F103851F0103941F0103B31F0103E8F
:1005200021F010E01093600000C1109360000F7084
:1005300003950093610010917A00112329F01017A0
:1005400019F010E010936000F0C0109160001038B6
:1005500019F0113839F00AC0139510936000009318
:100560006200E3C01A951093600010C0103919F0B2
:10057000113939F03BC0139510936000009362006D
:10058000D4C01A95109360000023F9F40091620022
:1005900010916500011719F41FEF10936500109179
:1005A0006400011749F4109165001F3F31F010936A
:1005B00064001FEF10936500B8C01FEF1093640034
:1005C00010E010939F00919AB0C0009363001091C7
:1005D000640010936500109162001093640011E0B4
:1005E00010939F001093A00091989FC0103B19F0AA
:1005F000113B39F081C013951093600000936200A5
:1006000094C01A951093600010916200AF93BF934D
:10061000103320F0103418F01035D0F064C0A1EE83
:10062000B0E0A10FB81D000F0C9310531770AFE886
:10063000B0E0A10FB81D0C91A7E9B0E0A10FB81D63
:100640000C93ABE6B0E0A10FB81D10E01C9351C0B5
:100650001054183020F11770A091780006FB10306C
:1006600011F4A0F919C0113011F4A1F915C012301C
:1006700011F4A2F911C0133011F4A3F90DC0143014
:1006800011F4A4F909C0153011F4A5F905C016300C
:1006900011F4A6F901C0A7F9A09378002AC0177039
:1006A000A091770006FB103011F4A0F919C01130A9
:1006B00011F4A1F915C0123011F4A2F911C01330D0
:1006C00011F4A3F90DC0143011F4A4F909C01530C8
:1006D00011F4A5F905C0163011F4A6F901C0A7F967
:1006E000A093770006C0A1EEB0E0A10FB81D000FE7
:1006F0000C93BF91AF9119C0103E19F0113E39F023
:1007000014C0139510936000009362000EC01A95F8
:100710001093600010916200110F110F001F00581C
:10072000109366000093670000C01F910F910FBFE8
:100730000F91579A18950F9302E30A95F1F70F91CD
:10074000089527B9369A0895349BFECF349A04B1A0
:1007500015B116950795169507950895222331F042
:100760002F93159507952A95E1F72F910895442326
:1007700041F04F9336952795179507954A95D1F7F0
:100780004F910895442341F04F93000F111F221FF2
:10079000331F4A95D1F74F910895019F8001089525
:1007A000379FE001279FA001179FD001079F902D41
:1007B000A10DB41FC51FD81D369FA001169F900D17
:1007C000A11DB41FC51FD81D269FA001069F802D07
:1007D000910DA41FB51FC81DD81D0A2F1B2F2C2F2C
:1007E0003D2F0895EE0FF0E0BB96EE0FFF1F059131
:1007F00015912591359108956F937F93E72FF2DF3F
:10080000802F912FA22FB32FE72FE395EBDF081B4B
:10081000190B2A0B3B0B8F939F93AF93BF93762FAC
:1008200060E04F93BDDF4F91BF91AF919F918F914A
:10083000080F191F2A1F3B1F7F916F91089540E0F9
:1008400002C07C5043957C30E0F70895EE0FFF1F07
:10085000E00FF81D04910895E00FF81DEE0FFF1F43
:10086000259134910895069506950695E5E8F0E002
:10087000F3DF00271127089560E0702F703718F01C
:10088000703938F00CC000E010E221E0E0E0F0E068
:100890000BC008E011E220E0ECE8FFE605C007EB42
:1008A0001DE121E0E7E6F2EE30E07ADF0E0F1F1FD8
:1008B0000895E199FECFBFB6F8942FBB1EBB0DBBC8
:1008C000E29AE19ABFBE0895E199FECFBFB6F894CF
:1008D0002FBB1EBBE09A0DB3BFBE08950027009347
:1008E0006B0000936C0000936D0000936E0000930A
:1008F0006F000093700000937100009372000091EC
:100900008F00009397000091900000939800009151
:100910009100009399000091920000939A00009139
:10092000930000939B000091940000939C00009121
:10093000950000939D000091960000939E000895FD
:10094000000F000F000F000F102F20E030E3BCDF7E
:10095000C1EED0E0C30FD81D088313953395303412
:10096000B1F700911F0100937700009120010093DF
:10097000780000917300009375000091740000935B
:100980007600ACDF0895CBE6D0E0C40FD81D2881F7
:1009900020FD14C0302FC7E9D0E0C40FD81D188146
:1009A000311B0AF43195353038F02160CBE6D0E0C8
:1009B000C40FD81D288302C010E0089511E00895E7
:1009C000F89400913400006804BF04BF0FE518E0FC
:1009D0000DBF1EBF882422243324442455246624BA
:1009E00077249924AA2422273327EE27FF2705E01E
:1009F0000093CD0000E00093610100936201009339
:100A000063010093640100937A00009379000093DE
:100A1000D90000939F000093A00000938B000093E7
:100A2000A8000093A9000093AA0000938D000093F2
:100A30008500009386000093870000936600009372
:100A400067000093E200009369000093E00002E079
:100A5000009388000FEF00936A000093DA00009380
:100A6000890000938A0000936400009365000EE5FE
:100A700014EB26E70093BC001093BD002093BE004A
:100A800000E010E020E00093BF001093C00020932E
:100A9000C1000FEF1FEF2FEF0093C2001093C300B0
:100AA0002093C40024E10093C5001093C600209356
:100AB000C70024E60093C8001093C9002093CA0021
:100AC00000E00093B0000093B5000093A7000093EE
:100AD0007B0000937C000093680000E00BBB00E00B
:100AE0000ABB0FEF08BB00E007BB00E005BB0FEF40
:100AF00004BB0CEF02BB0EEF01BB919A939A929844
:100B000000E003BF04E00EBD06E303BD0AE005BD3F
:100B100000E000BD0FE109B900E90AB906E806B92D
:100B200000E809BF789420918D000BDECFE8D0E07B
:100B3000C20FD81D09DE0883239503DEC39504DEAA
:100B400008832395FEDDC395FFDD08832395F9DD3A
:100B5000C395FADD08832395F4DDC395F5DD08839D
:100B60002395EFDDC395F0DD08832395EADDC3957A
:100B7000EBDD08832395E5DDC395E6DD088320E002
:100B800020938D00DEDD23E01EEF9EDED9DE23E024
:100B90001FEF9ADE00937A000CB51DB50093A100FB
:100BA0001093A2000CB51DB52091A1003091A200B8
:100BB000021B130B0A56184108F419C10091790061
:100BC000002329F0009363010FE300936201009179
:100BD00063010023D1F00091610110E4010F00389E
:100BE00030F0109162011A9541F0919A0AC010916B
:100BF00062011A9511F0919804C0919A00E0009357
:100C0000630100936101109362010CB51DB500935F
:100C1000A1001093A20000E111E020E130E040E0EB
:100C200050E0E2B3E06FE027E2BB85DDE6B3E0FF32
:100C3000312BE1FF322BE2FF412BE3FF422BE4FF9C
:100C4000512B110F220F000F61F702B3006F02BB8F
:100C500030937300409374005093790010916A00B0
:100C600010FF07C030937500409376001127109352
:100C70006A0000917300109175000117C9F120916D
:100C80007700EE27102710FF06C000FB20F90F9316
:100C900025DE0F91E0E111FF03C001FB21F9EFE038
:100CA00012FF03C002FB22F9EEE013FF03C003FBB7
:100CB00023F9EDE014FF03C004FB24F9E8E015FF7D
:100CC00003C005FB25F9E7E016FF03C006FB26F984
:100CD000E6E017FF03C007FB27F9E5E0E0936401B6
:100CE00010916301123011F020937700009375008A
:100CF00000917400109176000117B1F120917800F5
:100D0000EE27102710FF03C000FB20F9ECE011FFD5
:100D100003C001FB21F9EBE012FF03C002FB22F943
:100D2000EAE013FF03C003FB23F9E9E014FF03C06B
:100D300004FB24F9E4E015FF03C005FB25F9E3E01B
:100D400016FF03C006FB26F9E2E017FF03C007FB0E
:100D500027F9E1E0E093640110916301123011F092
:100D60002093780000937600109163011123F9F12C
:100D7000009164010023D9F1113029F1123031F0D2
:100D80000A9523E01EEF95DDDBDD27C01091DA0028
:100D9000112319F10A9523E01EEF8BDD10E010936B
:100DA000DA001093DB00000F000F000F000F00931C
:100DB000DC000091770000931F0100917800009300
:100DC00020018CDD0AC00395013109F401E00A9588
:100DD00000937A0023E01FEF6CDD919A00E000930E
:100DE000630100936101009362010093640100912B
:100DF000DA0007FD20C0E1991EC02091DB0010E35E
:100E0000120FC1EED0E0C10FD81D18810091DC0097
:100E1000020F30E03FBB0EBB1DBBBFB6F894E29A99
:100E2000E19ABFBE2F3021F023952093DB0003C051
:100E30001FEF1093DA0088DC20918D0020938E0044
:100E4000CFE8D0E0C20FD81D0883239527702093E8
:100E50008D0077DC40918E00403069F494DD1123E1
:100E600011F000931101009111010C3F08F00CEFFB
:100E700000931101A1C0413031F485DD112339F116
:100E80000093120199C0463099F47DDD112311F0D1
:100E900000931701009117010695025110F404E028
:100EA00004C0043008F001C004E00093D70084C0FF
:100EB000473071F468DD112311F00093180100919F
:100EC0001801DADC105800937B0010937C0074C08A
:100ED0003091770030FD0C949307423031F453DDAC
:100EE000112341F10093130125C0433041F44BDD40
:100EF0001123C1F000936800009314015DC04430D9
:100F000031F441DD1123D9F10093150138C045308A
:100F100049F439DD112331F00695102F1695010F94
:100F20000093160149C04230D9F42DDD112311F090
:100F300000931B0100911B013091780034FF08C021
:100F40003FEF30938300309382000093840034C0DD
:100F500030E03093830000938200009384002CC023
:100F6000433031F410DD112339F100931C0124C00A
:100F70004430D9F408DD112311F000931D010091D4
:100F80001D013091780034FF08C03FEF30937F009F
:100F900030937E00009380000FC030E030937F00DC
:100FA00000937E000093800007C0453029F4EBDCFD
:100FB000112311F000931E0100916300000F1091A6
:100FC0001501019F1092AF006CB57DB5262F372F0C
:100FD0000091A3001091A400601B710B2093A3004B
:100FE0003093A4006093A5007093A60000911301B4
:100FF000009539DC6091A5007091A600D1DB30919D
:10100000B1004091B2005091B3005058F0E0E0912F
:10101000B000EE23A1F46091C2007091C3008091F2
:10102000C400300F411F521F20F0361747075807E2
:10103000C8F0362F472F582FE1E0F1E013C0609140
:10104000BF007091C0008091C100301B410B520B5A
:1010500020F063177407850728F0362F472F582F85
:10106000E0E0F1E0E093B00050583093B1004093DD
:10107000B2005093B30000E010E020E0E091770070
:10108000E2FF09C0FF23B1F00091BC001091BD0048
:101090002091BE002F770093BF001093C0002093D3
:1010A000C1000095109520950093C2001093C300D5
:1010B0002093C4000091770002FF05C0FF2361F078
:1010C0005091BE0007C00091770003FF03C0550F89
:1010D0005FE7581D5093B400009114011091E20095
:1010E000011708F4012F009368000091170106957D
:1010F00006950095B8DB6091A5007091A60050DBC5
:101100003091B6004091B7005091B8005058F0E0CF
:10111000E091B500EE23A1F46091C8007091C90080
:101120008091CA00300F411F521F20F03617470729
:101130005807C8F0362F472F582FE1E0F1E013C0D1
:101140006091C5007091C6008091C700301B410BB3
:10115000520B20F063177407850728F0362F472FAE
:10116000582FE0E0F1E0E093B50050583093B6001E
:101170004093B7005093B80050585093D600109148
:10118000A70000911E01113069F000917E0012301D
:1011900049F000918000143029F060917F001330F5
:1011A00039F13AC060DB6091A5007091A600F8DAD1
:1011B0003091A8004091A9005091AA006091A70029
:1011C0006430D1F0623049F0300F411F521FF0F40B
:1011D0003FEF4FEF5FEF02E017C0301B410B520BA8
:1011E00078F060917F00651788F003E00093A70016
:1011F00033274427562F0AC0301B410B520B30F4C3
:1012000030E040E050E000E00093A7003093A800F9
:101210004093A9005093AA001091AB0000911C01CB
:10122000113069F000918200123049F00091840081
:10123000143029F060918300133039F13CC013DB86
:101240006091A5007091A600ABDA3091AC0040919E
:10125000AD005091AE006091AB006430D1F06230CF
:1012600049F0300F411F521F00F53FEF4FEF5FEF86
:1012700002E019C0301B410B520B78F060918300E3
:10128000651798F003E00093AB0033274427562FEF
:101290000CC0301B410B520B40F430E040E050E0FA
:1012A00000E00093E0000093AB003093AC0040936B
:1012B000AD005093AE0000919F00002371F404E054
:1012C0001091A700112351F10093A7001091AB00DA
:1012D000112321F10093AB0021C00091A000002355
:1012E000E9F000E00093A00000918800002319F0CD
:1012F0000A950093880001E00093A7000093AB00DB
:101300000093E0000FEF1FEF2FE70093B100109361
:10131000B2002093B30001E00093B00090E060E0E1
:10132000709164007F3F11F4AEC07C507136E8F7D5
:1013300001C0745F7432E8F37C5090918500A091F5
:101340008600B091870000918800002381F500910C
:10135000160189DA6F937F93622F732F00E010E0FC
:101360002091A5003091A60043E001DA19DA7F91BF
:101370006F91302F412F522F90918500A0918600C0
:10138000B09187006A177B0738F4931BA40BB50B49
:101390006A177B0750F006C0930FA41FB51F6A178A
:1013A0007B0718F490E0A62FB72F6A2F7B2F90931E
:1013B000850060938600709387000091660010910D
:1013C000670025E0CBD9202F312F020F131F020F0A
:1013D000131F600F711F70938C000091770007FF3F
:1013E0000C940F0A0091B4001091680020917700CE
:1013F00026FF10E0212F1695203810F01058120FFC
:101400000103800124E0AAD9600F711F77231AF429
:1014100060E070E004C07D3610F060E07CE66F9321
:101420007F93972F9D5008F49927969596959695BA
:101430009093D40004DAE0D9A5D91093CE0020937C
:10144000CF003093D0007F916F9100917B0010917D
:101450007C0024E083D9600F711F0091780001FDAA
:10146000745F972F9D5008F49927969596959695B9
:101470009093D500E4D9C0D985D91093D100209399
:10148000D2003093D300E0E0F0E00091770007FD58
:101490000C94570A0091B4001091680020917700D5
:1014A00026FF10E00103E12DF0E0111CFF0B00917D
:1014B000AE001091AF00019F8001001FE11FF81DD9
:1014C00000918C00000F00561BEA0103800120E010
:1014D00017FD2FEFE10FF21F0091120111270E0FE0
:1014E0001F1F112312F400E002C009F00FEF069550
:1014F000E5E4F0E0ABD9009389000A5008F400E07D
:1015000000938A001091110100918900003110F0C0
:10151000012F06C0E5E2F1E099D9011708F0012F8B
:101520000093DD000091AA00E5EAF0E08FD9009376
:101530008B000091BC001091BD002091BE0027FBE4
:1015400030F922FB40F934273695001F111F221F66
:101550000093BC001093BD002093BE0023CB8012EB
:1015600011151616161819191A1B1C1D1E1F2020DE
:10157000212223242526272728292A2B2C2D2D2EEE
:101580002F30313233343435363738393A3A3B3C00
:101590003D3E3F4041414243444546474748494A12
:1015A0004B4C4D4D4E4F5051525353545556575826
:1015B00059595A5B5C5D5E5F606061626364656639
:1015C000666768696A6B6C6D6D6E6F70717273734C
:1015D0007475767778797A7A7B7C7D7E7F8080805F
:1015E000818283848586868788898A8B8C8D8D8E7F
:1015F0008F90919293939495969798999A9A9B9C91
:101600009D9E9FA0A0A1A2A3A4A5A6A7A7A8A9AAA2
:10161000ABACADADAEAFB0B1B2B3B3B4B5B6B7B8B5
:10162000B9B9BABBBCBDBEBFBFC0C1C2C3C4C5C6C9
:10163000C6C7C8C9CACBCCCCCDCECFD0D1D2D3D3DC
:10164000D4D5D6D7D8D9D9DADBDCDDDEDFE0E0E1EE
:10165000E2E3E4E5E6E7E7E8EAEAEAEBEFEE801149
:1016600010151715161919191A1C1C1D1E1F1F20DD
:10167000222223242526262728292A2B2C2C2D2EEE
:101680002F3031323333343536373839393A3B3C01
:101690003D3E3F4040414243444546464748494A13
:1016A0004B4C4C4D4E4F5051525353545556575826
:1016B00059595A5B5C5D5E5F606061626364656638
:1016C000666768696A6B6C6D6D6E6F70717273734B
:1016D0007475767778797A7A7B7C7D7E7F8080805E
:1016E000818283848586868788898A8B8C8D8D8E7E
:1016F0008F90919293939495969798999A9A9B9C90
:101700009D9E9FA0A0A1A2A3A4A5A6A7A7A8A9AAA1
:10171000ABACADADAEAFB0B1B2B3B4B4B5B6B7B8B3
:10172000B9BABABBBCBDBEBFC0C0C1C2C3C4C5C6C6
:10173000C7C7C8C9CACBCCCDCDCECFD0D1D2D3D4D8
:10174000D4D5D6D7D8D9DADADBDCDDDEDEE0E1E1EC
:10175000E2E3E4E4E6E7E7E7EAEBE9EBF0EF801C3D
:10176000161414141516181A1B1C1D1D1E1E1F20DE
:1017700021222324252627272829292A2B2C2D2EF0
:101780002F30313232333435363738393A3A3B3C00
:101790003D3E3E3F40414243444546464748494A14
:1017A0004B4C4D4D4E4F5051525253545556575825
:1017B00059595A5B5C5D5E5F606161626364656537
:1017C000666768696A6B6C6D6D6E6F707172737449
:1017D000747576777879797A7B7C7D7E7F8080805E
:1017E000818283848586878788898A8B8C8C8D8E7D
:1017F0008F90919293939495969798999A9B9B9C8E
:101800009D9E9F9FA0A1A2A3A4A5A6A7A7A8A9AAA1
:10181000ABACADAEAEAFB0B1B2B3B3B4B5B6B7B8B2
:10182000B9BABABBBCBDBEBFC0C1C2C2C3C4C5C6C3
:10183000C6C7C8C9CACBCCCDCECECFD0D1D2D3D4D7
:10184000D5D6D7D7D8D9D9DADBDCDDDEDFE0E1E2E7
:10185000E2E3E3E4E5E6E8EAEBECECECEAE4800A58
:101860000F1A15131919171A1C1A1C1E1D1E2120D8
:10187000212323232526262829292A2C2C2C2E2EE9
:101880002F30313133343435373738393A3A3C3CFC
:101890003D3E3F3F41424243444546474748494A0F
:1018A0004B4C4D4D4E505051525353555556575821
:1018B000595A5B5B5C5D5E5F606161626364656633
:1018C000666769696A6B6C6C6E6E6F707172737447
:1018D0007475767778797A7A7B7C7D7E7F7F80815C
:1018E000818283848586868788898A8B8C8C8D8E7D
:1018F0008F90919292949495969797999A9A9B9C8F
:101900009D9E9F9FA0A1A2A3A4A5A5A6A7A8A9AAA2
:10191000ABABADADAEAFB0B0B2B3B3B4B5B6B7B8B4
:10192000B9B9BABBBCBDBEBEBFC1C1C2C3C4C4C6C7
:10193000C6C7C8C9C9CBCCCCCDCFCFD0D1D2D2D4D9
:10194000D4D4D6D7D7D8DADADBDDDDDDDFE0DFE2ED
:10195000E3E2E4E6E4E6E9E7E7EDEBE6F1F6800151
:101960001B131519141C161C191C1D1C201D211FCE
:10197000222223252427262828292B2A2D2C2E2EE7
:101980003030313232343436363738383A3A3C3CFB
:101990003D3E3F40404242434445464648484A4A0D
:1019A0004B4C4C4E4E50505152535454565657581F
:1019B000595A5A5C5C5D5E5F606062626364656632
:1019C0006668686A6A6B6C6D6E6E70707172737443
:1019D0007476767778797A7A7C7C7D7E7F80808059
:1019E000818283848486868788898A8A8C8C8D8E7E
:1019F0008F90909292939495969698989A9A9B9C91
:101A00009D9E9EA0A0A1A2A3A4A4A6A6A7A8A9AAA1
:101A1000AAACACADAEAFB0B0B2B2B4B4B5B6B6B8B5
:101A2000B8BABABBBCBDBEBEC0C0C1C2C3C4C4C6C6
:101A3000C6C8C8C9CACACCCCCECECFD0D0D2D2D4D8
:101A4000D3D6D5D7D8D8DAD9DCDBDDDEDEE1DFE3EB
:101A5000E0E4E3E4E7E4EAE4ECE7EBEDE5FF801A39
:101A600001181E11131D1B151A1F1B1A20211E1FE2
:101A7000242321242725252929282A2C2C2B2E2FE5
:101A80002E2F32323233353535383938393B3C3BFD
:101A90003D3F3E3F41424243454545474848494B0B
:101AA0004B4B4D4E4E4F5051515254555556585820
:101AB000585A5B5B5C5E5E5E606161626464646632
:101AC000676768696A6B6B6D6E6E6F717171737445
:101AD0007475777777797A7A7B7D7D7D7F8080805A
:101AE00081838383858686878989898B8C8C8D8F7A
:101AF0008F8F91929293959596979899999A9C9C8D
:101B00009C9E9F9FA0A2A2A2A4A5A5A6A8A8A8AAA1
:101B1000ABABACAEAFAFB0B1B2B2B3B5B5B5B7B8B1
:101B2000B8B9BBBBBBBDBEBEBFC1C2C1C3C5C4C5C6
:101B3000C7C8C7C8CBCBCBCDCECECED1D2D1D2D5D4
:101B4000D4D4D6D8D7D7DBDBD9DCDFDDDCE1E2DFEC
:101B5000E0E6E5E1E6EBE5E3EDEFE2E8FFE680391C
:101B60000B000D1D211B13131920211D1A1B2024EE
:101B7000242120222628282626282B2D2C2B2B2EEC
:101B80003132313031343636353537393B3B3A3BFB
:101B90003C3F40403F4042444545454547494A4A0D
:101BA0004A4B4D4E4F4F4F5052545454545658591F
:101BB00059595A5B5D5E5E5E5F6162636363646632
:101BC000676868686A6C6C6D6D6E6F717172727344
:101BD0007576777777787A7B7C7C7C7E7F80808057
:101BE00081828484848586888989898A8B8D8E8E7A
:101BF0008F8F91929393949496989898999A9C9D8C
:101C00009D9D9E9FA1A2A2A2A3A5A6A7A7A7A8AAA1
:101C1000ACACACACAEB0B1B1B1B2B3B5B6B6B6B7B0
:101C2000B9BBBBBBBBBCBEC0C1C0C0C1C4C5C6C5BF
:101C3000C5C7C9CBCBCACACCCFD0CFCECFD2D5D5D2
:101C4000D4D3D5D8DADAD8D8DADEE0DFDCDCE0E5E8
:101C5000E6E3DFE0E7EDEDE5DFE3F3FFF5C7805115
:101C6000290E02030C172024221D1815161A2024F1
:101C700026262421202124282B2C2C2B2A292A2CEF
:101C80002F323333333231323437393B3B3A3A3AFD
:101C90003B3D3F414242424242434547494A4A4A0C
:101CA0004A4A4B4C4E505152525152535456585925
:101CB0005A59595A5B5C5E60616161616263646636
:101CC0006869696969696A6C6E6F70717171717246
:101CD00074767778797979797A7C7D7F8080808055
:101CE00080818384868787878788898A8C8E8F8F77
:101CF0008F8F90919294969797979797989A9C9D8B
:101D00009E9F9F9F9FA0A2A4A5A6A7A7A6A7A8AA9B
:101D1000ACADAEAFAEAEAFB0B2B4B5B6B6B6B6B6A9
:101D2000B7B9BBBDBEBEBEBEBEBFC1C3C5C6C6C6BB
:101D3000C5C5C7C9CCCECFCECDCDCDCED1D4D6D7CB
:101D4000D6D5D4D4D5D8DCDFE0DFDCDADADCE0E6E7
:101D5000EAEBE8E3DEDCE0E9F4FDFEF2D7AF806118
:101D6000442B180B0403060C141C222628272522BA
:101D70001E1C1B1B1D2124282B2E2F2F2E2C2B2A03
:101D80002A2B2C2F31343638393939383737373810
:101D90003A3C3E4042444445444444444445474818
:101DA0004A4C4E4F50505050505051525355575925
:101DB0005A5B5C5C5C5C5C5C5D5E60616365666735
:101DC000686868686869696B6C6E70717374747444
:101DD000747475757677797A7C7E7F808080808058
:101DE00080808182848687898A8B8B8C8C8C8C8C7A
:101DF0008D8F9092949597979898989898999A9B88
:101E00009D9FA0A2A3A4A4A4A4A4A4A5A6A7A9AB93
:101E1000ADAEAFB0B0B0B0B0B0B1B2B4B6B8B9BB9F
:101E2000BCBCBCBCBCBBBCBCBEC0C2C4C6C8C9C9AF
:101E3000C9C8C7C7C7C8CACCCFD1D4D5D6D6D5D4C0
:101E4000D2D1D1D2D5D8DCDFE3E5E5E4E2DEDBD9DF
:101E5000D8DADEE4ECF4FAFDFCF5E8D5BC9F806D41
:101E60005A49382A1E140C08050506090D12181DBA
:101E700022262A2C2E2F2E2D2C2A292726252425D2
:101E80002627292C2F313437393B3C3D3D3D3D3D04
:101E90003C3B3B3B3B3B3C3D3F41434547494B4D36
:101EA0004E4F4F505050504F4F4F4F505052535431
:101EB00056585A5C5E5F6062626363636363636328
:101EC0006364646567686A6B6D6F7172747575764B
:101ED000767777777777777778797A7B7D7F808168
:101EE0008385868788898989898989898A8A8B8B6C
:101EF0008C8E8F9193959698999B9C9C9D9D9D9D72
:101F00009D9D9D9D9E9EA0A1A2A4A6A8AAACADAE9B
:101F1000B0B0B1B1B1B1B0B0B0B0B1B1B2B3B5B7AA
:101F2000B9BBBDBFC1C3C4C5C5C5C5C5C4C3C3C393
:101F3000C3C3C4C5C7C9CCCFD1D4D7D9DADBDCDBA6
:101F4000DAD9D7D6D4D3D2D1D2D4D6DADEE3E8EEFA
:101F5000F3F7FAFBFBF8F4ECE2D6C8B7A69380746B
:101F6000685B50453A3128201A140F0C0A080808FB
:101F7000090B0E1114181C2023272A2E3033353656
:101F800038383939383837363635343332323232F8
:101F90003333343537393B3D3F414345484A4C4D57
:101FA0004F5051525353535353535353535252520E
:101FB00053535454555658595B5C5E60626466676F
:101FC000696B6C6D6E6F707071717171717171711F
:101FD000717272727374747677787A7B7D7F808188
:101FE00083858688898A8C8C8D8E8E8E8F8F8F8F3D
:101FF0008F8F8F8F8F9090919293949597999A9CB1
:102000009EA0A2A4A5A7A8AAABACACADADAEAEAE47
:10201000ADADADADADADADADADAEAFB0B1B3B4B6D0
:10202000B8BBBDBFC1C3C5C7C9CBCCCDCDCECECE4D
:10203000CECDCCCBCACAC9C8C8C7C7C8C8CACBCD01
:10204000D0D2D6D9DDE0E4E8ECEFF2F5F7F8F8F815
:10205000F6F4F1ECE6E0D8CFC6BBB0A5988C80775B
:102060006E655D544C443C352F29231E1A161310FF
:102070000E0C0B0B0B0B0C0E101214171A1D202339
:1020800026292C2F3235373A3C3D3F4042434344CA
:10209000444444444443434242414141404040401F
:1020A000404141424344454648494B4D4F515355A9
:1020B00057595B5C5E6062636566676869696A6BF5
:1020C0006B6B6B6B6C6C6B6B6B6B6B6C6C6C6C6D58
:1020D0006D6E6F70717273757678797B7D7F80819C
:1020E000838587888A8B8D8E8F9091929393949419
:1020F0009494959595959594949595959595969791
:102100009798999A9B9D9EA0A2A4A5A7A9ABADAFB5
:10211000B1B3B5B7B8BABBBCBDBEBFBFC0C0C0C00D
:10212000C0BFBFBFBEBEBDBDBCBCBCBCBCBCBDBDDA
:10213000BEC0C1C3C4C6C9CBCED1D4D7DADDE0E3BB
:10214000E6E9ECEEF0F2F4F5F5F5F5F4F2F0EDEA8F
:10215000E6E2DDD7D1CBC4BCB4ACA39B928980E6C8
:10216000E7E5E4E5E6E5E5E5E5E5E5E5E5E5E5E51D
:10217000E5E5E5E5E5E5E5E5E5E5E5E5E5E5E5E50F
:10218000E5E5E5E5E5E5E5E5E5E5E5E5E5E5E5E5FF
:10219000E5E5E5E5E5E5E5E5E5E5E5E5E5E5E5E5EF
:1021A000E5E5E5E5E5E5E5E5E5E5E5E5E5E5E5E5DF
:1021B000E5E5E5E5E5E5E5E5E5E5E5E5E5E5E5E5CF
:1021C000E5E5E5E5E5E5E5E5E5E5E5E5E5E5E5E5BF
:1021D000E5E5E5E5E5E5E5E5E6E5E4E5E7E6801ADC
:1021E000191B1C1B1A1B1B1B1B1B1B1B1B1B1B1B41
:1021F0001B1B1B1B1B1B1B1B1B1B1B1B1B1B1B1B2F
:102200001B1B1B1B1B1B1B1B1B1B1B1B1B1B1B1B1E
:102210001B1B1B1B1B1B1B1B1B1B1B1B1B1B1B1B0E
:102220001B1B1B1B1B1B1B1B1B1B1B1B1B1B1B1BFE
:102230001B1B1B1B1B1B1B1B1B1B1B1B1B1B1B1BEE
:102240001B1B1B1B1B1B1B1B1B1B1B1B1B1B1B1BDE
:102250001B1B1B1B1B1B1B1B1A1B1C1B191A80E6A1
:10226000E8E4E4E6E6E4E5E6E5E4E5E5E5E5E5E51C
:10227000E5E5E5E5E5E5E5E5E5E5E5E5E5E5E5E50E
:10228000E5E5E5E5E5E5E5E5E5E5E5E5E5E5E5E5FE
:10229000E5E5E5E5E5E5E5E5E5E5E5E5E5E5E5E5EE
:1022A000E5E5E5E5E5E5E5E5E5E5E5E5E5E5E5E5DE
:1022B000E5E5E5E5E5E5E5E5E5E5E5E5E5E5E5E5CE
:1022C000E5E5E5E5E5E5E5E5E5E5E5E5E5E5E5E5BE
:1022D000E5E5E5E4E5E6E5E4E6E6E4E4E8E6801ADB
:1022E000181C1C1A1A1C1B1A1B1C1B1B1B1B1B1B40
:1022F0001B1B1B1B1B1B1B1B1B1B1B1B1B1B1B1B2E
:102300001B1B1B1B1B1B1B1B1B1B1B1B1B1B1B1B1D
:102310001B1B1B1B1B1B1B1B1B1B1B1B1B1B1B1B0D
:102320001B1B1B1B1B1B1B1B1B1B1B1B1B1B1B1BFD
:102330001B1B1B1B1B1B1B1B1B1B1B1B1B1B1B1BED
:102340001B1B1B1B1B1B1B1B1B1B1B1B1B1B1B1BDD
:102350001B1B1B1C1B1A1B1C1A1A1C1C181A80DDA9
:10236000E3E5E6E7E7E6E6E5E5E4E4E5E5E5E6E618
:10237000E6E6E5E5E5E5E5E5E5E5E5E6E5E5E5E50A
:10238000E5E5E5E5E5E5E5E5E5E5E5E5E5E5E5E5FD
:10239000E5E5E5E5E5E5E5E5E5E5E5E5E5E5E5E5ED
:1023A000E5E5E5E5E5E5E5E5E5E5E5E5E5E5E5E5DD
:1023B000E5E5E5E5E5E5E5E5E5E5E5E5E5E5E5E5CD
:1023C000E5E6E5E5E5E5E5E5E5E5E5E6E6E6E6E5B8
:1023D000E5E5E4E4E5E5E6E6E7E7E6E5E3DD8023D9
:1023E0001D1B1A19191A1A1B1B1C1C1B1B1B1A1A42
:1023F0001A1A1B1B1B1B1B1B1B1B1B1A1B1B1B1B30
:102400001B1B1B1B1B1B1B1B1B1B1B1B1B1B1B1B1C
:102410001B1B1B1B1B1B1B1B1B1B1B1B1B1B1B1B0C
:102420001B1B1B1B1B1B1B1B1B1B1B1B1B1B1B1BFC
:102430001B1B1B1B1B1B1B1B1B1B1B1B1B1B1B1BEC
:102440001B1A1B1B1B1B1B1B1B1B1B1A1A1A1A1BE1
:102450001B1B1C1C1B1B1A1A19191A1B1D2380ED90
:10246000EAE0E5E8E3E4E7E4E4E6E5E4E6E5E4E51C
:10247000E6E4E5E6E4E5E6E5E5E5E5E4E5E5E4E50D
:10248000E5E4E5E5E5E5E5E5E5E5E5E5E5E5E5E5FD
:10249000E5E5E5E5E5E5E5E5E5E5E5E5E5E5E5E5EC
:1024A000E5E5E5E5E5E5E5E5E5E5E5E5E5E5E5E5DC
:1024B000E5E5E5E5E5E5E5E5E5E5E5E4E5E5E4E5CE
:1024C000E5E4E5E5E5E5E6E5E4E6E5E4E6E5E4E5BD
:1024D000E6E4E5E6E4E4E7E4E3E8E5E0EAED8013DA
:1024E00016201B181D1C191C1C1A1B1C1A1B1C1B3C
:1024F0001A1C1B1A1C1B1A1B1B1B1B1C1B1B1C1B2B
:102500001B1C1B1B1B1B1B1B1B1B1B1B1B1B1B1B1A
:102510001B1B1B1B1B1B1B1B1B1B1B1B1B1B1B1B0B
:102520001B1B1B1B1B1B1B1B1B1B1B1B1B1B1B1BFB
:102530001B1B1B1B1B1B1B1B1B1B1B1C1B1B1C1BE9
:102540001B1C1B1B1B1B1A1B1C1A1B1C1A1B1C1BDA
:102550001A1C1B1A1C1C191C1D181B20161380F595
:10256000DFE6E7E2E8E1E8E3E5E5E4E7E3E6E4E522
:10257000E5E4E6E4E6E4E5E5E4E6E4E6E4E5E5E50D
:10258000E5E4E6E4E5E5E5E5E4E6E4E5E5E5E5E4FE
:10259000E5E4E5E5E5E5E4E5E4E5E5E5E5E4E5E4F0
:1025A000E5E5E5E5E4E5E4E5E5E5E5E4E5E4E5E5DF
:1025B000E5E5E4E6E4E5E5E5E5E4E6E4E5E5E5E5CD
:1025C000E4E6E4E6E4E5E5E4E6E4E6E4E5E5E4E6BD
:1025D000E3E7E4E5E5E3E8E1E8E2E7E6DFF5800BE1
:1025E000211A191E181F181D1B1B1C191D1A1C1B34
:1025F0001B1C1A1C1A1C1B1B1C1A1C1A1C1B1B1B29
:102600001B1C1A1C1B1B1B1B1C1A1C1B1B1B1B1C17
:102610001B1C1B1B1B1B1C1B1C1B1B1B1B1C1B1C05
:102620001B1B1B1B1C1B1C1B1B1B1B1C1B1C1B1BF6
:102630001B1B1C1A1C1B1B1B1B1C1A1C1B1B1B1BE8
:102640001C1A1C1A1C1B1B1C1A1C1A1C1B1B1C1AD8
:102650001D191C1B1B1D181F181E191A210B80DEAB
:10266000F6E2DDE9E9E1E3E9E6E2E5E8E4E3E7E60D
:10267000E3E4E7E5E3E5E7E4E4E6E6E4E5E6E5E40C
:10268000E5E6E4E4E6E6E4E5E6E5E4E5E6E4E4E6FA
:10269000E5E4E5E6E5E4E5E6E4E4E6E5E4E5E6E5EB
:1026A000E4E5E6E4E4E6E5E4E5E6E5E4E5E6E4E4DD
:1026B000E6E5E4E5E6E5E4E6E6E4E4E6E5E4E5E6C9
:1026C000E5E4E6E6E4E4E7E5E3E5E7E4E3E6E7E3BB
:1026D000E4E8E5E2E6E9E3E1E9E9DDE2F6DE8022CD
:1026E0000A1E2317171F1D171A1E1B181C1D191A47
:1026F0001D1C191B1D1B191C1C1A1A1C1B1A1B1C28
:102700001B1A1C1C1A1A1C1B1A1B1C1B1A1C1C1A19
:102710001B1C1B1A1B1C1B1A1C1C1A1B1C1B1A1B08
:102720001C1B1A1C1C1A1B1C1B1A1B1C1B1A1C1CF6
:102730001A1B1C1B1A1B1C1A1A1C1C1A1B1C1B1AEA
:102740001B1C1A1A1C1C191B1D1B191C1D1A191DD8
:102750001C181B1E1A171D1F1717231E0A2280C1C3
:10276000ECF7EDDFDBE2EAECE7E1E0E4E9E9E5E202
:10277000E2E5E8E8E5E3E3E6E8E7E4E3E4E6E7E604
:10278000E4E3E4E6E7E6E4E3E5E6E7E5E4E4E5E7F9
:10279000E6E5E4E4E5E7E6E5E4E4E6E7E6E4E4E4E8
:1027A000E6E7E6E4E4E5E6E7E5E4E4E5E6E7E5E4D4
:1027B000E4E5E7E6E5E3E4E6E7E6E4E3E4E6E7E6C6
:1027C000E4E3E4E7E8E6E3E3E5E8E8E5E2E2E5E9B7
:1027D000E9E4E0E1E7ECEAE2DBDFEDF7ECC1803FC2
:1027E00014091321251E1614191F201C17171B1E50
:1027F0001E1B18181B1D1D1A18191C1D1C1A191A2E
:102800001C1D1C1A191A1C1D1B1A191B1C1C1B1918
:102810001A1B1C1C1B191A1B1C1C1A191A1C1C1C09
:102820001A191A1C1C1B1A191B1C1C1B1A191B1CFD
:102830001C1B191A1B1D1C1A191A1C1D1C1A191AEB
:102840001C1D1C19181A1D1D1B18181B1E1E1B17DA
:10285000171C201F1914161E25211309143F80ABC5
:10286000D0E9F6F7F0E7DFDBDDE2E8EBECEAE6E201
:10287000E0E1E3E7E9EAE9E6E3E2E2E4E6E8E9E801
:10288000E6E4E3E3E4E6E7E8E8E6E4E3E3E4E5E7F7
:10289000E8E8E6E5E3E3E4E5E7E8E8E7E5E4E3E4E0
:1028A000E5E7E8E8E7E5E4E3E3E5E6E8E8E7E5E4CB
:1028B000E3E3E4E6E8E8E7E6E4E3E3E4E6E8E9E8BE
:1028C000E6E4E2E2E3E6E9EAE9E7E3E1E0E2E6EAB8
:1028D000ECEBE8E2DDDBDFE7F0F7F6E9D0AB8055C3
:1028E00030170A0910192125231E181514161A1E4F
:1028F000201F1D191716171A1D1E1E1C1A1817182F
:102900001A1C1D1D1C1A1918181A1C1D1D1C1B1918
:1029100018181A1B1D1D1C1B191818191B1C1D1C0F
:102920001B191818191B1C1D1D1B1A1818191B1C04
:102930001D1D1C1A1818191A1C1D1D1C1A181718F1
:102940001A1C1E1E1D1A171617191D1F201E1A16D7
:102950001415181E2325211910090A173055809CBB
:10296000B7CEE0EEF6F8F7F2ECE6E1DDDCDCDFE234
:10297000E6E9ECEDEDEBE9E6E3E1E0E0E2E3E6E8F1
:10298000E9EAEAEAE8E6E4E3E2E2E2E4E5E7E9E9E3
:10299000EAE9E8E6E5E3E2E2E3E4E5E7E8E9E9E9D4
:1029A000E8E7E5E4E3E2E2E3E5E6E8E9EAE9E9E7C6
:1029B000E5E4E2E2E2E3E4E6E8EAEAEAE9E8E6E3BB
:1029C000E2E0E0E1E3E6E9EBEDEDECE9E6E2DFDCB5
:1029D000DCDDE1E6ECF2F7F8F6EEE0CEB79C8064E1
:1029E000493220120A08090E141A1F232424211E1A
:1029F0001A1714131315171A1D1F20201E1D1A183D
:102A000017161616181A1C1D1E1E1E1C1B1917172A
:102A10001617181A1B1D1E1E1D1C1B191817171719
:102A200018191B1C1D1E1E1D1B1A18171617171907
:102A30001B1C1E1E1E1D1C1A1816161617181A1DF2
:102A40001E20201F1D1A1715131314171A1E2124D8
:102A500024231F1A140E09080A1220324964809098
:102A60009FAFBDCAD6E0E8EFF4F7F9FAF9F7F4F151
:102A7000EDEAE6E3E1DEDDDCDCDDDEDFE1E4E6E835
:102A8000EAECEDEEEFEFEEEDECEAE9E7E5E3E2E1AB
:102A9000E0E0E0E1E2E3E4E6E7E9EAECEDEDEDEDCC
:102AA000EDECEAE9E7E6E4E3E2E1E0E0E0E1E2E3DD
:102AB000E5E7E9EAECEDEEEFEFEEEDECEAE8E6E46F
:102AC000E1DFDEDDDCDCDDDEE1E3E6EAEDF1F4F7BB
:102AD000F9FAF9F7F4EFE8E0D6CABDAF9F9080703D
:102AE000615143362A2018110C09070607090C0FFB
:102AF00013161A1D1F222324242322211F1C1A18F7
:102B00001614131211111213141617191B1D1E1F60
:102B10002020201F1E1D1C1A19171614131313131F
:102B200013141617191A1C1D1E1F2020201F1E1DEE
:102B30001B191716141312111112131416181A1C3C
:102B40001F212223242423221F1D1A16130F0C09D0
:102B5000070607090C1118202A3643516170808935
:102B6000939DA6AFB8C0C8D0D7DDE3E8EDF1F4F788
:102B7000F9FBFCFCFCFBFAF9F8F6F4F1EFEDEAE8FE
:102B8000E6E4E2E0DFDEDDDCDCDCDCDDDDDEE0E156
:102B9000E2E4E6E7E9EBECEEEFF0F1F2F3F3F3F366
:102BA000F3F2F1F0EFEEECEBE9E7E6E4E2E1E0DE90
:102BB000DDDDDCDCDCDCDDDEDFE0E2E4E6E8EAED06
:102BC000EFF1F4F6F8F9FAFBFCFCFCFBF9F7F4F191
:102BD000EDE8E3DDD7D0C8C0B8AFA69D9389807774
:102BE0006D635A514840383029231D18130F0C09C2
:102BF0000705040404050607080A0C0F111316182C
:102C00001A1C1E2021222324242424232322201FB3
:102C10001E1C1A191715141211100F0E0D0D0D0D83
:102C20000D0E0F101112141517191A1C1E1F202239
:102C3000232324242424232221201E1C1A181613A3
:102C4000110F0C0A080706050404040507090C0FF8
:102C500013181D232930384048515A636D778086F8
:102C60008D939AA0A7ADB3B9BFC4CACFD4D9DDE1C3
:102C7000E5E9EDF0F2F5F7F9FBFCFEFEFFFFFFFFE3
:102C8000FFFFFEFDFCFBF9F8F6F5F3F1EFEDECEAE2
:102C9000E8E6E5E3E2E0DFDEDDDCDBDBDADADADA48
:102CA000DADBDBDCDDDEDFE0E2E3E5E6E8EAECED03
:102CB000EFF1F3F5F6F8F9FBFCFDFEFFFFFFFFFF78
:102CC000FFFEFEFCFBF9F7F5F2F0EDE9E5E1DDD9F9
:102CD000D4CFCAC4BFB9B3ADA7A09A938D86807A6A
:102CE000736D666059534D47413C36312C27231F85
:102CF0001B1713100E0B0907050402020101000146
:102D000001010203040507080A0B0D0F1113141625
:102D1000181A1B1D1E20212223242525262626269F
:102D200026252524232221201E1D1B1A18161413C4
:102D3000110F0D0B0A080705040302010101000130
:102D4000010202040507090B0E1013171B1F23278E
:102D50002C31363C41474D535960666D737A807E05
:102D60007C7A78767472706E6C6A68666462605E93
:102D70005C5A58565452504E4C4A48464442403E83
:102D80003C3A38363432302E2C2A28262422201E73
:102D90001C1A18161412100E0C0A0806040200025F
:102DA0000406080A0C0E10121416181A1C1E2022F3
:102DB0002426282A2C2E30323436383A3C3E4042E3
:102DC0004446484A4C4E50525456585A5C5E6062D3
:102DD0006466686A6C6E70727476787A7C7E8082C3
:102DE0008486888A8C8E90929496989A9C9EA0A2B3
:102DF000A4A6A8AAACAEB0B2B4B6B8BABCBEC0C2A3
:102E0000C4C6C8CACCCED0D2D4D6D8DADCDEE0E292
:102E1000E4E6E8EAECEEF0F2F4F6F8FAFCFEFFFE87
:102E2000FCFAF8F6F4F2F0EEECEAE8E6E4E2E0DED2
:102E3000DCDAD8D6D4D2D0CECCCAC8C6C4C2C0BEC2
:102E4000BCBAB8B6B4B2B0AEACAAA8A6A4A2A09EB2
:102E50009C9A98969492908E8C8A88868482807EA2
:102E60007C7A78767472706E6C6A68666462605E92
:102E70005C5A58565452504E4C4A48464442403E82
:102E80003C3A38363432302E2C2A28262422201E72
:102E90001C1A18161412100E0C0A0806040201025D
:102EA0000406080A0C0E10121416181A1C1E2022F2
:102EB0002426282A2C2E30323436383A3C3E4042E2
:102EC0004446484A4C4E50525456585A5C5E6062D2
:102ED0006466686A6C6E70727476787A7C7E8082C2
:102EE0008486888A8C8E90929496989A9C9EA0A2B2
:102EF000A4A6A8AAACAEB0B2B4B6B8BABCBEC0C2A2
:102F0000C4C6C8CACCCED0D2D4D6D8DADCDEE0E291
:102F1000E4E6E8EAECEEF0F2F4F6F8FAFCFEFFFE86
:102F2000FCFAF8F6F4F2F0EEECEAE8E6E4E2E0DED1
:102F3000DCDAD8D6D4D2D0CECCCAC8C6C4C2C0BEC1
:102F4000BCBAB8B6B4B2B0AEACAAA8A6A4A2A09EB1
:102F50009C9A98969492908E8C8A88868482807EA1
:102F60007C7A78767472706E6C6A68666462605E91
:102F70005C5A58565452504E4C4A48464442403E81
:102F80003C3A38363432302E2C2A28262422201E71
:102F90001C1A18161412100E0C0A0806040201025C
:102FA0000406080A0C0E10121416181A1C1E2022F1
:102FB0002426282A2C2E30323436383A3C3E4042E1
:102FC0004446484A4C4E50525456585A5C5E6062D1
:102FD0006466686A6C6E70727476787A7C7E8082C1
:102FE0008486888A8C8E90929496989A9C9EA0A2B1
:102FF000A4A6A8AAACAEB0B2B4B6B8BABCBEC0C2A1
:10300000C4C6C8CACCCED0D2D4D6D8DADCDEE0E290
:10301000E4E6E8EAECEEF0F2F4F6F8FAFCFEFFFE85
:10302000FCFAF8F6F4F2F0EEECEAE8E6E4E2E0DED0
:10303000DCDAD8D6D4D2D0CECCCAC8C6C4C2C0BEC0
:10304000BCBAB8B6B4B2B0AEACAAA8A6A4A2A09EB0
:103050009C9A98969492908E8C8A88868482807EA0
:103060007C7A78767472706E6C6A68666462605E90
:103070005C5A58565452504E4C4A48464442403E80
:103080003C3A38363432302E2C2A28262422201E70
:103090001C1A18161412100E0C0A0806040201025B
:1030A0000406080A0C0E10121416181A1C1E2022F0
:1030B0002426282A2C2E30323436383A3C3E4042E0
:1030C0004446484A4C4E50525456585A5C5E6062D0
:1030D0006466686A6C6E70727476787A7C7E8082C0
:1030E0008486888A8C8E90929496989A9C9EA0A2B0
:1030F000A4A6A8AAACAEB0B2B4B6B8BABCBEC0C2A0
:10310000C4C6C8CACCCED0D2D4D6D8DADCDEE0E28F
:10311000E4E6E8EAECEEF0F2F4F6F8FAFCFEFFFE84
:10312000FCFAF8F6F4F2F0EEECEAE8E6E4E2E0DECF
:10313000DCDAD8D6D4D2D0CECCCAC8C6C4C2C0BEBF
:10314000BCBAB8B6B4B2B0AEACAAA8A6A4A2A09EAF
:103150009C9A98969492908E8C8A88868482807E9F
:103160007D7A78767472706E6C6A68666462605E8E
:103170005C5A58565452504E4C4A48464442403E7F
:103180003C3A38363432302E2C2A28262422201E6F
:103190001C1A18161412100E0C0A0806040201025A
:1031A0000406080A0C0E10121416181A1C1E2022EF
:1031B0002426282A2C2E30323436383A3C3E4042DF
:1031C0004446484A4C4E50525456585A5C5E6062CF
:1031D0006466686A6C6E70727476787A7D7E8082BE
:1031E0008386888A8C8E90929496989A9C9EA0A2B0
:1031F000A4A6A8AAACAEB0B2B4B6B8BABCBEC0C29F
:10320000C4C6C8CACCCED0D2D4D6D8DADCDEE0E28E
:10321000E4E6E8EAECEEF0F2F4F6F8FAFCFEFFFE83
:10322000FCFAF8F6F4F2F0EEECEAE8E6E4E2E0DECE
:10323000DCDAD8D6D4D2D0CECCCAC8C6C4C2C0BEBE
:10324000BCBAB8B6B4B2B0AEACAAA8A6A4A2A09EAE
:103250009C9A98969492908E8C8A88868382807E9F
:103260007D7B78767572706E6C6A68666462605E8B
:103270005C5A58565452504E4C4A48464442403E7E
:103280003C3A38363432302E2C2A28262422201E6E
:103290001C1A18161412100E0C0A08070402010258
:1032A0000407080A0C0E10121416181A1C1E2022ED
:1032B0002426282A2C2E30323436383A3C3E4042DE
:1032C0004446484A4C4E50525456585A5C5E6062CE
:1032D0006466686A6C6E70727576787B7D7E8082BB
:1032E0008385888A8B8E90929496989A9C9EA0A2B1
:1032F000A4A6A8AAACAEB0B2B4B6B8BABCBEC0C29E
:10330000C4C6C8CACCCED0D2D4D6D8DADCDEE0E28D
:10331000E4E6E8EAECEEF0F2F4F6F8F9FCFEFFFE83
:10332000FCF9F8F6F4F2F0EEECEAE8E6E4E2E0DECE
:10333000DCDAD8D6D4D2D0CECCCAC8C6C4C2C0BEBD
:10334000BCBAB8B6B4B2B0AEACAAA8A6A4A2A09EAD
:103350009C9A98969492908E8B8A88858382807F9F
:103360007D7A78767473716E6C6A68676462605E89
:103370005C5B58565452504E4C4A48464442403E7C
:103380003C3A38363432302E2C2A28262422211E6C
:103390001C1A18171512100E0C0B09060402020253
:1033A0000406090B0C0E10121517181A1C1E2122E8
:1033B0002426282A2C2E30323436383A3C3E4042DD
:1033C0004446484A4C4E50525456585B5C5E6062CC
:1033D0006467686A6C6E71737476787A7D7F8081B9
:1033E0008386888A8C8D8F92949698999C9EA0A2B1
:1033F000A4A5A8AAACAEB0B2B4B6B8BABCBEC0C29E
:10340000C4C6C8CACCCED0D2D4D6D8DADCDEDFE28D
:10341000E4E6E8E9EBEEF0F2F4F5F7FAFCFEFEFE86
:10342000FCFAF7F5F4F2F0EEEBE9E8E6E4E2DFDED1
:10343000DCDAD8D6D4D2D0CECCCAC8C6C4C2C0BEBC
:10344000BCBAB8B6B4B2B0AEACAAA8A5A4A2A09EAD
:103450009C99989694928F8D8C8A88868381807FA0
:103460007D7B79767472706E6D6B69676462605E85
:103470005C5B59575552504E4C4A49474543403E74
:103480003C3A38363533312E2C2A28262423211F66
:103490001C1A18161413110F0D0A08060403020350
:1034A0000406080A0D0F11131416181A1C1F2123E5
:1034B0002426282A2C2E31333536383A3C3E4043D8
:1034C0004547494A4C4E50525557595B5C5E6062C5
:1034D0006467696B6D6E70727476797B7D7F8081B5
:1034E0008385878A8C8E9092939597999C9EA0A2B3
:1034F000A4A5A7A9ABAEB0B2B4B6B7B9BBBDC0C2A4
:10350000C4C6C8CACBCDCFD2D4D6D8DADCDDDFE191
:10351000E4E6E8EAECEDEFF1F3F6F8FAFCFDFEFD87
:10352000FCFAF8F6F3F1EFEDECEAE8E6E4E1DFDDD2
:10353000DCDAD8D6D4D2CFCDCBCAC8C6C4C2C0BDBF
:10354000BBB9B7B6B4B2B0AEABA9A7A5A4A2A09EB2
:103550009C9997959392908E8C8A87858381807EA3
:103560007C7A78767472716F6D6B69676462605E85
:103570005C5A58565553514F4D4B48464442403E75
:103580003C3A39373533312F2C2A28262422201E65
:103590001D1B19171513100E0C090706040403044C
:1035A000040607090C0E10131517191B1D1E2022E7
:1035B0002426282A2C2F31333537393A3C3E4042D5
:1035C0004446484B4D4F51535556585A5C5E6062C5
:1035D0006467696B6D6F71727476787A7C7E8082B5
:1035E0008486888A8C8E8F91939597999C9EA0A2B1
:1035F000A4A6A8AAABADAFB1B3B5B8BABCBEC0C2A1
:10360000C4C6C7C9CBCDCFD1D4D6D8DADCDEE0E290
:10361000E3E5E7E9EBEDF0F2F4F7F9FAFCFCFDFC89
:10362000FCFAF9F7F4F2F0EDEBE9E7E5E3E2E0DECE
:10363000DCDAD8D6D4D1CFCDCBC9C7C6C4C2C0BEC0
:10364000BCBAB8B5B3B1AFADABAAA8A6A4A2A09EB0
:103650009C99979593918F8E8C8A88868482807EA0
:103660007C7A78767472706E6C6A68676563615F85
:103670005D5B59575553514E4C4A48464442403E73
:103680003C3A38363533312F2D2B29272523211F5E
:103690001C1A181513110F0D0B090807060606064C
:1036A000060708090B0D0F111315181A1C1F2123EB
:1036B0002527292B2D2F31333536383A3C3E4042D1
:1036C0004446484A4C4E51535557595B5D5F6163C0
:1036D0006567686A6C6E70727476787A7C7E8082B8
:1036E0008486888A8C8E9092949698999B9D9FA1AF
:1036F000A3A5A7A9ABADAFB2B4B6B8BABCBEC0C2A1
:10370000C4C6C8CACBCDCFD1D3D5D7D9DBDDDFE195
:10371000E4E6E8EBEDEFF1F3F5F7F8F9FAFAFAFA87
:10372000FAF9F8F7F5F3F1EFEDEBE8E6E4E1DFDDC8
:10373000DBD9D7D5D3D1CFCDCBCAC8C6C4C2C0BEC2
:10374000BCBAB8B6B4B2AFADABA9A7A5A3A19F9DB3
:103750009B9998969492908E8C8A88868482807E9B
:103760007C7A787673716F6D6B6967656361605E93
:103770005C5A5857555351504E4C4A484644424063
:103780003E3C3A373533302E2C29272522201E1C6B
:103790001917151412100F0D0C0B0A0A0909090943
:1037A000090A0A0B0C0D0F1012141517191C1E20F4
:1037B000222527292C2E303335373A3C3E404244CF
:1037C00046484A4C4E5051535557585A5C5E6061BA
:1037D000636567696B6D6F717376787A7C7E8082C2
:1037E0008486888A8D8F91939597999B9D9FA0A29F
:1037F000A4A6A8A9ABADAFB0B2B4B6B8BABCBEC0AF
:10380000C2C4C6C9CBCDD0D2D4D7D9DBDEE0E2E486
:10381000E7E9EBECEEF0F1F3F4F5F6F6F7F7F7F78E
:10382000F7F6F6F5F4F3F1F0EEECEBE9E7E4E2E0BD
:10383000DEDBD9D7D4D2D0CDCBC9C6C4C2C0BEBCC2
:10384000BAB8B6B4B2B0AFADABA9A8A6A4A2A09FB7
:103850009D9B99979593918F8D8A88868482807F8E
:103860007D7B7A78767473716F6D6B696765636160
:103870005F5D5B59575452504D4B494644423F3D62
:103880003A383633312F2C2A28262422201E1C1A9F
:1038900019171614131211100F0F0E0E0D0D0D0D1A
:1038A0000D0E0E0F0F10111213141617191A1C1EDD
:1038B00020222426282A2C2F313336383A3D3F4205
:1038C0004446494B4D50525457595B5D5F616365A7
:1038D00067696B6D6F71737476787A7B7D7F808199
:1038E000838586888A8C8D8F91939597999B9D9FD0
:1038F000A1A3A5A7A9ACAEB0B3B5B7BABCBEC1C3AE
:10390000C6C8CACDCFD1D4D6D8DADCDEE0E2E4E650
:10391000E7E9EAECEDEEEFF0F1F1F2F2F3F3F3F3B5
:10392000F3F2F2F1F1F0EFEEEDECEAE9E7E6E4E2D2
:10393000E0DEDCDAD8D6D4D1CFCDCAC8C6C3C1BE8A
:10394000BCBAB7B5B3B0AEACA9A7A5A3A19F9D9BC8
:0E39500099979593918F8D8C8A8886858381B7
:00000001FF
